:100000000AC023C022C021C020C01FC01EC01DC006
:100010001CC01BC01AC011241FBECFEDCDBF10E005
:10002000A0E6B0E0E4E7F7E003C0C89531960D9292
:10003000A238B107D1F710E0A2E8B0E001C01D92EC
:10004000AE38B107E1F781D294C3DACFCF93DF9313
:10005000CDB7DEB724970FB6F894DEBF0FBECDBF85
:100060009C838B8313C080E392E09A83898305C0CD
:1000700089819A8101979A83898389819A810097DE
:10008000B9F78B819C8101979C838B838B819C81A9
:10009000009749F724960FB6F894DEBF0FBECDBF88
:1000A000DF91CF910895CF93DF93CDB7DEB7E8E32B
:1000B000F0E01082E7E3F0E08FE18083E2E3F0E03C
:1000C0001082E1E3F0E08AE58083DF91CF9108952B
:1000D000CF93DF93CDB7DEB722970FB6F894DEBF8C
:1000E0000FBECDBFA2E3B0E0E2E3F0E08081806428
:1000F0008C9388E390E09A83898305C089819A81F3
:1001000001979A83898389819A810097B9F7A2E33D
:10011000B0E0E2E3F0E090818FEB89238C932296AC
:100120000FB6F894DEBF0FBECDBFDF91CF9108951B
:10013000CF93DF93CDB7DEB7A2E3B0E0E2E3F0E028
:1001400090818FEE89238C938EE690E07FDFE8E349
:10015000F0E083E08083BCDF8AE090E077DFE8E3D3
:10016000F0E083E08083B4DF8AE090E06FDFE8E3D3
:10017000F0E083E08083ACDF8AE090E067DFE8E3D3
:10018000F0E082E08083A4DFDF91CF910895CF93E8
:10019000DF93CDB7DEB721970FB6F894DEBF0FBE61
:1001A000CDBF898382E090E051DF898182958F7095
:1001B00099279093830080938200A8E3B0E0E8E35E
:1001C000F0E08081282F207F809182009091830031
:1001D000822B8C93A2E3B0E0E2E3F0E080818061C7
:1001E0008C9376DF898199278F709070909383002C
:1001F00080938200A8E3B0E0E8E3F0E08081282F5C
:10020000207F8091820090918300822B8C93A2E3C7
:10021000B0E0E2E3F0E0808180618C9359DF2196C9
:100220000FB6F894DEBF0FBECDBFDF91CF9108951A
:10023000CF93DF93CDB7DEB721970FB6F894DEBF2B
:100240000FBECDBF898382E090E000DF8981829577
:100250008F7099279093830080938200A8E3B0E089
:10026000E8E3F0E08081282F207F80918200909148
:100270008300822B8C93A2E3B0E0E2E3F0E0908174
:100280008FEE89238C9324DF898199278F7090705A
:100290009093830080938200A8E3B0E0E8E3F0E06D
:1002A0008081282F207F8091820090918300822B73
:1002B0008C93A2E3B0E0E2E3F0E090818FEE89233B
:1002C0008C9306DF21960FB6F894DEBF0FBECDBF2C
:1002D000DF91CF910895CF93DF93CDB7DEB722970B
:1002E0000FB6F894DEBF0FBECDBFA8E3B0E0E8E3E1
:1002F000F0E080818F7180628C93A7E3B0E0E7E348
:10030000F0E080818F7180628C93E6E3F0E0808181
:10031000992780749070009729F081E090E09A838B
:10032000898302C01A82198289819A8122960FB626
:10033000F894DEBF0FBECDBFDF91CF910895CF936C
:10034000DF93CDB7DEB722970FB6F894DEBF0FBEAE
:10035000CDBFA8E3B0E0E8E3F0E080818F71806476
:100360008C93A7E3B0E0E7E3F0E080818F718064D5
:100370008C93E6E3F0E0808188232CF481E090E028
:100380009A83898302C01A82198289819A8122966E
:100390000FB6F894DEBF0FBECDBFDF91CF910895A9
:1003A000CF93DF93CDB7DEB722970FB6F894DEBFB9
:1003B0000FBECDBFA8E3B0E0E8E3F0E08081982F66
:1003C0009F7180E8892B8C93A7E3B0E0E7E3F0E02E
:1003D0008081982F9F7180E8892B8C93E6E3F0E071
:1003E0008081992780729070009729F081E090E0D9
:1003F0009A83898302C01A82198289819A812296FE
:100400000FB6F894DEBF0FBECDBFDF91CF91089538
:10041000CF93DF93CDB7DEB722970FB6F894DEBF48
:100420000FBECDBFA8E3B0E0E8E3F0E080818F71BC
:1004300080648C93A7E3B0E0E7E3F0E080818F7104
:1004400080648C93E6E3F0E080819927807290705D
:10045000009729F081E090E09A83898302C01A8294
:10046000198289819A8122960FB6F894DEBF0FBE59
:10047000CDBFDF91CF910895CF93DF93CDB7DEB796
:1004800022970FB6F894DEBF0FBECDBFA8E3B0E051
:10049000E8E3F0E08081982F9F7180E8892B8C93AE
:1004A000A7E3B0E0E7E3F0E08081982F9F7180E858
:1004B000892B8C93E6E3F0E080819927807490701B
:1004C000009729F081E090E09A83898302C01A8224
:1004D000198289819A8122960FB6F894DEBF0FBEE9
:1004E000CDBFDF91CF910895CF93DF93CDB7DEB726
:1004F00022970FB6F894DEBF0FBECDBFA8E3B0E0E1
:10050000E8E3F0E080818F7180628C93A7E3B0E034
:10051000E7E3F0E080818F7180628C93E6E3F0E0A6
:10052000808188232CF481E090E09A83898302C043
:100530001A82198289819A8122960FB6F894DEBFB9
:100540000FBECDBFDF91CF910895CF93DF93CDB78D
:10055000DEB762970FB6F894DEBF0FBECDBFA3DD46
:10056000E7DD81E080938B000DC080918B0099279F
:10057000F92FE82FEC57FF4F108280918B008F5F8F
:1005800080938B0080918B00873078F38CE050DE75
:1005900081E04EDE00C09FDE282F33273A8B298B67
:1005A00080918500188A1F86882321F481E090E0DD
:1005B000988B8F8789899A892F85388982239323FD
:1005C0000097E1F081E034DE80E832DE10928B00AB
:1005D0000EC080918B009927F92FE82FE05AFF4F2A
:1005E0008081D5DD80918B008F5F80938B0080911F
:1005F0008B00803170F381E0809385006CDE1E8675
:100600001D86882321F481E090E09E878D8780916C
:10061000850099272D853E8582239323009711F02D
:10062000109285008CDE282F33273C872B87809102
:1006300086001A861986882321F481E090E09A8743
:1006400089878B859C8529853A858223932300970A
:1006500099F181E0EDDD80E8EBDD10928B000EC0BA
:1006600080918B009927F92FE82FE05AFF4F808166
:100670008EDD80918B008F5F80938B0080918B004B
:10068000803170F380ECD4DD10928B000EC080912D
:100690008B009927F92FE82FEF58FF4F808177DDE6
:1006A00080918B008F5F80938B0080918B008031D5
:1006B00070F381E08093860042DE18861F828823D3
:1006C00021F481E090E098878F83809186009927BC
:1006D0002F81388582239323009711F01092860092
:1006E000CBDE282F33273E832D83809189001C8207
:1006F0001B82882321F481E090E09C838B838D8191
:100700009E812B813C81822393230097E1F081E03D
:100710008FDD80EC8DDD10928B000EC080918B0000
:100720009927F92FE82FEF58FF4F808130DD809116
:100730008B008F5F80938B0080918B00803170F3F2
:1007400081E08093890098DE1A821982882321F43F
:1007500081E090E09A83898380918900992729819B
:100760003A8182239323009709F415CF10928900D0
:0407700012CFFFCFD6
:1007740020202020204156522D4D5420202020207E
:1007840000206F6C696D65782E636F6D2F646576DC
:02079400200043
:00000001FF
